:020000040000FA
:040000004BEF00F0D2
:0400080004EF04F00D
:080018000CEF04F0A4A8FED7D0
:100020006D6E12006BA202D06B986B88A4AAFED7EB
:100030006E501200A68EA69CA684A688550EA76EAA
:10004000AA0EA76EA682000001EE00F0080E016E57
:10005000A68EA69CA6840A00080E006EEECFF5FFC1
:100060000F00002EFBD7550EA76EAA0EA76EA68214
:100070000000012EF1D7A6943F0EF65E000EF75A4F
:10008000000EF85A400E006E0900F5500EEC00F01C
:10009000002EFAD7120084BE00EF04F0070EB46EF3
:1000A000000E896E000E8A6E400E8B6E000E8C6EF6
:1000B0000C0E8D6E000E8E6E020E8F6EFF0E926E07
:1000C000FF0E936EBF0E946EFF0E956E330E966EFE
:1000D000FF0E976EFD0E986E0F0EC16E0C0EAF6E7A
:1000E000AC84AC8AAB88AB8E0C0E6F6E6C846C8A61
:1000F0006B886B8EFE0EF66EFF0EF76E3F0EF86E7F
:100100000800F5CF05F0053A05420542030E051635
:10011000200E036EF80E046E030E0518D8A404D04A
:10012000200E036EFA0E046E020E0518D8A404D039
:10013000200E036EFC0E046E010E0518D8A404D028
:10014000200E036EFD0E046E000EF66E080EF76EA6
:10015000000EF86E12EC00F0420AFCE112EC00F026
:100160006F0A02E06F0AF8D712EC00F06F0A02E0A3
:100170006F0AF2D712EC00F0740A02E0740AECD7AE
:1001800012EC00F04C0A02E04C0AE6D712EC00F048
:100190006F0A02E06F0AE0D712EC00F0610A02E099
:1001A000610ADAD712EC00F0640A02E0640AD4D7DC
:1001B00005500EEC00F001EE00F0400E026E12EC65
:1001C00000F0EE6E022EFBD71AEC00F0033EF3D7E0
:1001D000043EF1D7A69EA69CA684100E036EAA6AC2
:1001E000A96A01EE00F0400E026E12EC00F0EE6E15
:1001F000022EFBD7400E006E01EE00F0EECFA8FFFE
:10020000550EA76EAA0EA76EA6820000A6B2FED754
:10021000A94AAA2A002EF2D7400EA95E000EAA5AB9
:10022000400E006EA6800000A8500EEC00F0A94A17
:10023000AA2A002EF7D7032ED4D7A69412EC00F0EA
:100240004F0E0EEC00F04B0E0EEC00F08D8CFFD735
:02080000FFD720
:020808001000DE
:020818001000CE
:020000040030CA
:06000100061600F38381E6
:06000800FF80FF80FF00F5
:0200000400F00A
:10000000FFFFFFFFFFFFFFFFFFFFFFFFFFFFFFFF00
:10001000FFFFFFFFFFFFFFFFFFFFFFFFFFFFFFFFF0
:10002000FFFFFFFFFFFFFFFFFFFFFFFFFFFFFFFFE0
:10003000FFFFFFFFFFFFFFFFFFFFFFFFFFFFFFFFD0
:00000001FF
